:030000000219FDE5
:03000B000200AA46
:03002B000201626D
:03005B000202EAB4
:030073000202D0B6
:1000800002030406080C10182030406080040608A3
:100090000C10182030406080A0C000070F1F3F0DDB
:1000A0000D04050D050205030302C2AFC0D0C0E078
:1000B000206217E5256002E473E525F4F58A758B67
:1000C00000D262D0E0D0D0D2AF3285268AC262E5BB
:1000D00026F46030758B00D0E0D0D0C295C294C2B7
:1000E00093D2AF32C295C294C293206E0D20660A9D
:1000F0007405D5E0FDE57EF45290758B00D0E0D01C
:10010000D0D2AF32758A00C28DD26201FA01B93005
:100110006805206602D29501B9306805206602D2D2
:100120009401B9306805206602D29301B9D29230A9
:10013000680A2066077403D5E0FDD29501B9D29113
:1001400030680A2066077403D5E0FDD29401B9D265
:1001500090D29230680A2066077403D5E0FDD293EE
:1001600001B9C2AFC2AD53E6EFC0D0C0E0D2D3D226
:10017000AFC2CEE52A6007207449152A21C3780052
:10018000790020742EE580307E01F430E70278FF9C
:1001900053DACF207E0343DA20307E0343DA10C2E5
:1001A000D8C271E580307E01F430E70279FFC3E800
:1001B0009970CB306103752A18207403752A18884A
:1001C0005FD27020740DE52B6004152B21D343DA28
:1001D00001C2D82070024131A85F206102C27020A4
:1001E00074367982B70431C3E894F0400374F0F8B0
:1001F000E8C4540F28F87984B703024118C313C325
:10020000138721200802C313200A06C3C898F841A7
:100210001828F8500374FFF88822E52D5406601161
:10022000E533C313C31324062522F5225003752298
:10023000FF7882B6044E852224A824C3E524956461
:100240004002A864C3E895664002A8668825E5696F
:1002500070024182C3E8AA699A5003E8FAE4F9EA15
:10026000C333FBE56BF45B29400D256AF8E56A6052
:1002700002156A400B41820AC3E56A9A5002056A78
:1002800078FF8826C3E52594404002D26420CF0A37
:10029000D0E0D0D043E610D2AD32C2CF053A7801DB
:1002A000E52A6005307402152AC3E55F9401400514
:1002B00075620041C6756300756C00E5622401F546
:1002C0006250037562FFD0E0D0D043E610D2AD3269
:1002D000C2AFC0D053E67FC2607591008556948549
:1002E0005795759104D0D0D2AF32C2AF53E6EFC26A
:1002F000ADC0D0C0E0C0F0D2D3D2AFA8FBA9FCC241
:10030000D8307102615153DACF207E0343DA1030C6
:100310007E0343DA20D271E580307E01F420E702CB
:10032000612888278928A17E53DACF207E0343DA0B
:1003300020307E0343DA10C2D8C271307402A16A41
:100340007800E580307E01F430E702A16A885FA181
:100350005253DACF207E0343DA20307E0343DA1093
:10036000C271206102812A53DACF207E0343DA1062
:10037000307E0343DA20C2D8D271885A895BC3E841
:100380009558F8E99559F97B007E087A00C3E894FE
:100390008CE994005005755E00811C882178A2E6E6
:1003A000A8216055C3E894C8E994005008E4D2E459
:1003B000FB7A0A61F7C3E89468E994015008E4D233
:1003C000E3FB7A0F61F7C3E894D0E994025008E4A4
:1003D000D2E2FB7A1E61F7C3E894A0E994055008C5
:1003E000E4D2E1FB7A3C61F7C3E89498E9940850C1
:1003F00008E4D2E0FB7A787E00C3E8955CFCE995DE
:100400005DFD30E70AECF42401FCEDF43400FD75E9
:100410005E00C3EC9AED9E5003755E01885C895DB9
:10042000855A58855B597802A152C3E89527F8E9A7
:100430009528F9307C02A136307B02A136307A0251
:10044000A12F207502814DE9FDE8FC816CE9C31301
:10045000F9E813F8307902A12FE9C313F9E813F88A
:10046000307802A12FE9C313FDE813FC20612CC3EF
:0F047000EC941CED940240028183ED701EC3ECEE
:10047F0094C850180529E52970021529C3E5299458
:10048F000A5002A16A755F00D270A16AE529600265
:10049F0015297888E6F97400207F087896B9030249
:1004AF00789EE624FAFEE43400FFC3EC9EFCED9F39
:1004BF00FD9208B90310A2085007207609D2768161
:1004CF00D5307602C276A2085016B9030DECF4248B
:1004DF0001FCEDF43400FD0204EF78007900A13641
:1004EF00B90315EC33FCED33FDC3EC940AFCED942A
:1004FF0000FD50047C007D00C3EC94FFED940040A0
:10050F000678FF7900A136EC8575F0A4C5F0A2F747
:10051F0033F87900400302055278FF790002055243
:10052F00E9C313F9E813F8307C0EE9600278FFC3D2
:10053F00E81338F8E43400F9C3E894FFE994004075
:10054F000278FF885FD270206102A16A741FF45590
:10055F002F4BF52FC274EB7002D274752A183074BA
:10056F0003752A0A306102A17E20740353DAFE203C
:10057F007403752B06D0F0D0E0D0D0D2AD43E61087
:10058F003279010205AE79030205AE790A0205AE92
:10059F00791E0205AE79640205AE79C80205AE7800
:1005AF0017E4D5E0FDD8FAD9F6227A147B78020544
:1005BF00D57A107B8C0205D57A0D7BB40205D57ADE
:1005CF000B7BC80205D57902B27DE4D291D5E0FD4F
:1005DF00D294D5E0FDC294D5E0FDC291D5E0FDD215
:1005EF0095E576D5E0FDC2957496D5E0FDD9D9EAAB
:1005FF00F8D5E0FDD8FBDBCED29122C37C007D0085
:10060F0075F00005F0EA33FAEB33FB50F6EB13FB12
:10061F00EA13FAC3E9FFE8FEE89AF8E99BF95004F8
:10062F00EFF9EEF8B3EC33FCED33FDD5F0DFEDF978
:10063F00ECF822E889F08A20D2D4F8A9F07B0030B8
:10064F00F70B7BFFF42401F8E9F43400F9E8852077
:10065F00F0A4ADF0F8E98520F0A4AFF0FEED2EF98F
:10066F0074003FFA7C04C3EA13FAE913F9E813F8AC
:10067F00DCF48BF030F70AE8F42401F8E9F43400E5
:10068F00F9E889F0C2D4F8A9F0227882B6040302FF
:10069F0006F4C3E55F940140030206BE852224E4FD
:1006AF00F545F546F547F548F549C26D0206F4786C
:1006BF0082E6FCD26DE522F523783879C7AA40ABE4
:1006CF0041C3EB13FBEA13FAEC146013C3EB13FBF8
:1006DF00EA13FAEC14146007C3EB13FBEA13FAD115
:1006EF000A8845894622C3E5459523F8E5469400D7
:1006FF00F9500CC3E89480E994FF4016020725C314
:10070F00E8947FE994005003020725787F7900026F
:10071F000725788079FF884A894B22E54A2547F8D3
:10072F00E54B3548F9854B20E4300701F43549FA9C
:10073F0030E709C3EA94F04015020763C3EA940F48
:10074F00500302076378FF79FF7A0F02076378007F
:10075F0079007AF0C3E5249564500AC37401952497
:10076F00500B020781E54B20E70E020781E54B3066
:10077F00E706884789488A492278A4E6FAC3E54AFA
:10078F0033F8E54B33F9D142E930E70BC3E89480F6
:10079F00E994FF4013E1BBC3E8947FE99400500252
:1007AF00E1BB787F7900E1BB788079FFE820E7151E
:1007BF00C3E52398F84009C3E8940140030207E218
:1007CF0078010207E2E8F424012523F84003020729
:1007DF00E278FF884C2278A5E6FAA848A949D142C9
:1007EF00E930E70CC3E89401E994FF4016020816BC
:1007FF00C3E894FFE99400500302081678FF7900CC
:10080F00020816780179FFE920E715C3E54C98F83F
:10081F004009C3E89401400302083D780102083DF6
:10082F00E8F42401254CF8400302083D78FF8824A2
:10083F002278FFC26420693D206A12D264C3E54169
:10084F00940A4009C3E52594405002C26479A1E798
:10085F006023E541601F74FF8541F0848539F030D6
:0F086F006A0375F005A4F8C5F0600278FFC3E8CE
:10087E0095675002A867886622C3E5409440E5411B
:10088E009401E5665003140198046002F566220295
:10089E0008A02275E890227883E6FFE5E820ECF7C1
:1008AE00A8BDA9BE0573C3E57394084052757300C5
:1008BE00E9FA79A0E76044EA7007E574601B020864
:1008CE00DBC3E895746010E5745006600C140208E2
:1008DE00E70460F90208E7E574F574C3946D401BF4
:1008EE007564C0C394044013756480C39404400BB4
:1008FE00756440C39404400375640075BB0622E51D
:10090E00642410500274FFF5647982B70402213416
:10091E00C3A864E524985002A824C3E89566400253
:10092E00A86688258826E573B4070375BB10227464
:10093E003279A687F0A4C5F0A2F733F8C3E8956420
:10094E004002A86488228824882588268867227514
:10095E0040007541F022C2AF75C820A8CCA9CDAA1F
:10096E003A30CF010A75C824D2AFAB3BAC3C883BC2
:10097E00893CC3E89BF8E99C206908F9306702417D
:10098E007921D6AD3D8A3DF9EA9DFA600478FF796A
:10099E00FFAE3EAF3F8B3E8C3FC3EC9FFCC3E99C4A
:1009AE00F542A83BA93CC3E89EF8E99FF9C3E5418F
:1009BE0013FBE54013FAE82AF540E93BF5415006F2
:1009CE007540FF7541FF4120AA40AB41AC40AD419F
:1009DE007E047F02C3EB940440021E1FC3EB9408F7
:1009EE0040021E1FC3ED13FDEC13FCDEF7C3EA9CA1
:1009FE00FAEB9DFBEF6009C3E913F9E813F8DFF793
:100A0E00EA28FAEB39FB8A408B4150067BFF8B407C
:100A1E008B41C3EB94025002D2673069047F0341CD
:100A2E004B7892E6FFC3E537948240110FC3E5374A
:100A3E0094A040010FC3EF940640027F057E04E5AB
:100A4E0041C4540FF9E541C454F0F8E540C4540FC5
:100A5E0028F8C3E89EFAE99400FB4009C3EA940221
:100A6E00EB940050047A02E4FB41C5AA40AB41EB83
:100A7E00C4FEEAC4540F4EFCC3EA9CFAEB9400FB8E
:100A8E00C3E813C313F8EA28FAEB3400FB8A408B51
:100A9E0041C3EB94024002C2677804EBC4FE7B00B4
:100AAE00EAC4540F4EFAC3EA98FA4005C3940250B2
:100ABE00027A027892E6FF30600241C58552568571
:100ACE005357D26043E680C3E49AF8E49BF930674B
:100ADE0002615FE8FAE9FBD3E913FDE813FC8852E3
:100AEE008953C3EF94036038EF20E00DE82CF8E94A
:100AFE003DF9ECFAEDFB020B1AE828F8E939F9C3D7
:100B0E00E82402F8E93400F97AFE7BFFC3EF940380
:100B1E00400E8A548B55884E894F8C508D5161935F
:100B2E00885489558A4E8B4F8C508D51306920C315
:100B3E00E53394034019E542A2E713F8E555F42492
:100B4E000138400B20E7087554FFF42401F5556178
:100B5E0093E8FAD3E813FC8852C3EF94036020EFB6
:100B6E0020E007E82CF8ECFA617FE8282402F87AF6
:100B7E00FEC3EF940340088A54884E8C50619388CC
:100B8E00548A4E8C50E56BC3335002646BF56B3058
:100B9E006002619D753402D26043E680E52D5406F5
:100BAE006026A840A941C3E913F9E813F8C2AF5370
:100BBE00E67F759100C3E498F594E499F5957591E7
:100BCE0004D26043E680D2AF22D265754400752010
:100BDE0000306B03752040020BF6D265754400752C
:100BEE002040306B03752000D2AF7801206722E5DC
:100BFE002D54066002C265C3E54194054013780288
:100C0E00940540087803940540027806306902780E
:100C1E000A206019E544601530690AC3E533940370
:100C2E004003D53406D2AFD26C81C771A5D2AF00C6
:100C3E0000C2AF206726E541C3FB940F40027B0F35
:100C4E00EB240530730123306A02742820620123DD
:100C5E00F93069027982E58BC39940B50544E59B6D
:0F0C6E005440B5200281B130690A08C3E8940AE6
:100C7D00400108811F20650261F6C26553E67F754C
:100C8D0091003067107594007595FE759104D260D2
:100C9D0043E68061F6AE40AF41C3E49EF594E49F18
:100CAD00F5958198C3E5339402500261F6306502E3
:100CBD0061F6D80281C5811FC26C53E67F75910024
:100CCD00855494855595759104854E56854F57D20B
:100CDD006043E680D2AFE52D54066008206A020518
:100CED0033020D01306C0D206B0A2065071581153F
:100CFD008102156F2278003064053065027801E5B8
:100D0D003775F007A4F9E5F028F5F0E9A2F013A284
:100D1D00F113A2F213F537C394785003753778C3E6
:100D2D00E53795384008D266C295C294C2933060BB
:100D3D0002A13B855056855157D26043E680222053
:100D4D007D11C2AF754302D291C292D2AF759F1180
:100D5D00020F23C2AF754302D291C290D2AF759FDD
:100D6D0011020F23307245207D22C2AF75430390CF
:100D7D00013E757E02C293D290D292306204D2941B
:100D8D00A191C291D2AF759F01020F23C2AF7543DE
:100D9D000390013E757E02C295D292306204D294C8
:100DAD00A1B1C291D2AF759F21020F23207D17C231
:100DBD00AF754303900119C293306202D294D2AF42
:100DCD00759F01020F23C2AF754303900119C295A0
:100DDD00306202D294D2AF759F21020F23207D1174
:100DED00C2AF754304D292C290D2AF759F21020F4C
:100DFD0023C2AF754304D290D292C292D2AF759FE7
:100E0D0001020F23307243207D20C2AF7543059040
:100E1D00012D757E04C294D291306204D295C12FFA
:100E2D00C292D2AF759F11020F23C2AF75430590C9
:100E3D00014F757E01C294D291306204D293C14F9D
:100E4D00C290D2AF759F11020F23207D17C2AF75CF
:100E5D00430590010FC294306202D295D2AF759FB7
:100E6D0011020F23C2AF754305900123C294306266
:100E7D00EBD293D2AF759F11020F23207D13C2AF1A
:100E8D00754306D290D292C291D2AF759F01020FD7
:100E9D0023C2AF754306D292C291D2AF759F210284
:100EAD000F23307244207D20C2AF75430190014F56
:100EBD00757E01C295D292306204D293C1CDC2909B
:100ECD00D2AF759F21020F23C2AF75430190012D43
:100EDD00757E04C293D290D292306204D295C1EF46
:100EED00C292D2AF759F01E123207D16C2AF75432B
:100EFD0001900123C295306202D293D2AF759F212A
:100F0D00E123C2AF75430190010FC293306202D24B
:100F1D0095D2AF759F01C2662290010D757E00C2FC
:100F2D0095C294C293D292D291D290C2622278800D
:100F3D0076090876090876040876FF0876030876A0
:100F4D00FF08760A087601087601087601788C7616
:100F5D00010876FF0876FF0876FF0876FF0876FF12
:100F6D000876030876FF0876FF0876FF08762508D1
:100F7D0076D00876280876500876040876FF08762D
:100F8D000208760008767A0876FF08760108760161
:100F9D00087600087603227887E6FFC2727888E625
:100FAD00C394036008C27DE630E102D27DC27E7833
:100FBD0089E630E102D27EC3EF94026008758E019E
:100FCD00D273020FD7758E00C273227880E614900B
:100FDD0000809378A4F67881E6149000809378A52C
:100FED00F67886E61490008D9378A6F6789CE675D3
:100FFD0038FF75390CB402067538A075390AB4037B
:10100D000675388275390578A3E61490009A93F524
:10101D0069120F2622227896E6FA7897E6FB7888F1
:10102D00E6B40305C3EB940EFB307F047A007BFF1F
:10103D00C3EB9AFCC3948250027C827575000575D2
:10104D00EC8575F0A4C3E5F0947D40F222D27F11BA
:10105D002312059F7A007B007C10120595E55F2A0F
:0F106D00FA74003BFBDCF37C04C3EB13FBEA13C8
:10107C00FADCF7FEC27F112322E5EF20E603752090
:10108C00000520903FFFE520146006901DFF1460C2
:10109C00009304600375EF1253D9BF7581C043FFF1
:1010AC008012059075EF0243B203E5B3240420E7E8
:1010BC000DF521E5E320E0068521B343E301120F92
:1010CC00267580FF75A40075F19075D47F75908797
:1010DC0075A5BF75F2BF75D50075A60175E241E423
:1010EC00F8F6D8FD756B01120F3B1215B178988686
:1010FC0076753001C2AF1205A91205B912059F12FF
:10110C0005C012059F1205C712059FC2AF78FA7968
:10111C00FA308707D9FBD8F7021C00120FA4120F64
:10112C00D81122112378988676120F26758850755F
:10113C00891275C82475910475D84075A82275B8A4
:10114C000275E690759B80759D0075D10E75BC5827
:10115C0075BB0675BA1175E880120590D2AF1208EE
:10116C009D53DACF207E0343DA20307E0343DA101E
:10117C0043DA01C2D8C2711205A9D2617B037A0C81
:10118C00E55E70077A0CDB0302111712059F2070C5
:10119C0003021117C270E55FC3940240E1E52F54BE
:1011AC001F856160F561B560D5DAD5C26153DACFC0
:1011BC00207E0343DA20307E0343DA10C2D8C2719A
:1011CC0078A2E67008D274E52F54E0F52FC275753D
:1011DC0029001205A4307409C3E529940A4002D2EF
:1011EC007512059578023074027800C3E55F98405B
:1011FC00F0C2AF1205B91205B91205B9D2AF12057A
:10120C00A9754D007888E6B4030241EE1205957875
:10121C008CE6C3940150030212EEE530C3940150E6
:10122C00030212EE207435C3E55F94FF50030212E3
:10123C00EEC2AF1205CED2AF1205A4C3E55F940186
:10124C0050EFC2AF1205B912059A1205B9D2AF12FE
:10125C0005A4C3E55F94FF40E90217597F02D27FD2
:10126C0011231205A4C2AFC27F1123AE5FC3E55F89
:10127C00947FD2AF4076120590C2AF1205CED2AF9A
:10128C00DFDC115AC3EE94057897F61205A91215F6
:10129C00F31216DC7F0AD27F11231205A4C2AFC24F
:1012AC007F1123AE5FC3E55F947FD2AF50E612058A
:1012BC0090C2AF1205B912059A1205B9D2AFDFD69A
:1012CC00115AEE24057896F61205A91215F3121789
:1012DC000B1205A41123C3E55F94FF5002413002A9
:1012EC001759C3E55F954D4003855F4D1205A478F2
:1012FC00017988E7B403027805C3E55F98400241A1
:10130C0010C2AF1205CE1205CE1205CED2AF120509
:10131C00A9753000E4F531F5320531E531F4703959
:10132C000532789AE67819146012783214600D78C8
:10133C007D14600878FA146003753200C3E53298A6
:10134C00401715327531B478998676C2AF1205CE36
:10135C00D2AF789886761205A412059AE52A700504
:10136C00307402211778012074027806C3E55F9867
:10137C0040A77888E6C3940360031205A4E52A709D
:10138C0003021117C2AF120F26E4F522F523F52440
:10139C00F525F526F56AD2AF7885E6C333F568E412
:1013AC00F545F546F547F548F549F573F52CF52D5A
:1013BC00F53775730875BB101205901208A1E5E896
:1013CC0020ECFBA8BDA9BEE97001F888741208A531
:1013DC0075730875BB107887E6FE7602120FA47839
:1013EC0087EEF6C2AF7564FF12093D852264852233
:1013FC0065852266D2AF75220175240175250175AC
:10140C00260185636C756D017888E6B40307C27D8F
:10141C00307602D27DD268D269753300120E8812F2
:10142C000EAF12095D12096412095D1209641209EA
:10143C005D02144DC2AF120FA4D2AF75730075BB11
:10144C0006120BE8120699120D02120D4C120964C9
:10145C00120BD7306D031206F520670312084030CB
:0E146C006703120887120D02120D7112096437
:10147A00120BE8306D0312072A120D02120DEA123E
:10148A000964120BD7306D03120788120D02120E6F
:10149A0011120964120BE8306D031207E5120D02EE
:1014AA00120E881209641208A1120BD7120D021229
:1014BA000EAF1208A5120964306935206B328567B0
:1014CA006485676585636C756D0179187A0CC3E567
:1014DA003399400FC269D26A8A358567648567661F
:1014EA000214FAC3E55F9401400302144D02157712
:1014FA00306A1B206B18E535147004C26A8140F506
:10150A0035C3E55F9401400302144D021577753621
:10151A0000C3E56278FA985054307404E52A604DA5
:10152A007888E6B40317207D05207607A147307630
:10153A0002A147206B07D26B856764818C78F030F3
:10154A006B058567647820C3E541985002814D3068
:10155A006B1BC26BC27D307602D27DD26A753512A0
:10156A00856764814D0536E55F6002A17A753600AC
:10157A00C2AF120F267887E6FE7602120FA478878A
:10158A00EEF6E4F522F523F524F525F526F568C2ED
:10159A0068D2AF120590120F26307409C3E536944B
:1015AA0005400221176120901A0D7820121635E5A0
:1015BA0020B4550CA3121635E520B4AA030215D39C
:1015CA00120F3B1215F30215F2901A0378807B0A68
:1015DA00121635A308DBF9901A0F788C7B181216AD
:1015EA0035A308DBF9901A2722C2AF121674121615
:1015FA004E901A00740E12163AA3740412163AA3E5
:10160A00741412163A901A0378807B0A121639A3B8
:10161A0008DBF9901A0F788C7B18121639A308DBAD
:10162A00F9121687121665901A2722E493F622E613
:10163A00438F01538FFD75EF0275B7A575B7F1F0AA
:10164A00538FFE22438F02438F0175EF0275B7A5B0
:10165A0075B7F1901A0DF0538FFC22901A0D74553C
:10166A00D13A901A0E74AAD13A227A3079D07820D7
:10167A00901A40D135E520F709A3DAF7227A3079B2
:10168A00D0901A40E7D13A09A3DAF922AB77A878C1
:10169A00BB01027980BB02027981BB03027982BB5A
:1016AA0004027984BB05027986BB06027992BB07DC
:1016BA00027987BB080279A3BB0902799CBB0A029B
:1016CA007988BB0B027989E8F7227C051205A9DC27
:1016DA00FB22C2AF1205B91205C01205C71205CE08
:1016EA0012059A1205B91205C01205C71205CE12C3
:1016FA00059A1205B91205C01205C71205CED2AF56
:10170A0022C2AF1205CE1205C71205C01205B912C0
:10171A00059A1205CE1205C71205C01205B912059F
:10172A009A1205CE1205C71205C01205B9D2AF2208
:10173A00AE77AF78C2AF1205B91205B91205B91260
:10174A00059ADEF21205CE12059ADFF8D2AF22D13F
:10175A00DCD1D4D1D4757701757801757900F13A65
:10176A007C05AD5F1205A9C3ED955F70F5C3E55F12
:10177A009401400AC3E55F94FF4032021795D1965F
:10178A00B1F3D1DCC2AF75EF12D1D4DCD50579C380
:10179A00E5799403500280C6D1D40578E577149090
:1017AA00009F93F808C3E57898500280AED1D4D14F
:1017BA00D40577C3E577940C5002809C120F3BB195
:0817CA00F3C2AF75EF12D1D498
:0319FD0002108550
:101A00000E0414090904FF03FF0A01010155AA018C
:101A1000FFFFFFFFFF03FFFFFF25D0285004FF0259
:081A2000007AFF01010003FF41
:101A400023585032354123202020202020202020E0
:101A500023424C48454C4923463333302320202031
:101A60002020202020202020202020202020202076
:101C0000C2AFC2D353D9BF7581C043B20343FF8073
:101C1000752438752503B1C975EF0275E24043F1AB
:101C20008053A47F75D400D2877DFA780379E67C4F
:101C300010752200752300901DD67B0675249875BB
:101C400025013087028142208708D8FBD9F9DCF7CB
:101C500081B4308708D8FBD9F9DCF781B4B189E4C5
:101C600093A3C39A6004DDC381B4DBDBB17B600264
:101C7000812B7B08E493FAA3B15CDBF87A30B15C8A
:101C8000752200752300B17BEAFCEBFDC3ED94FEE9
:101C9000400EB17B8A278B28ED30E0048A828B834B
:101CA000B17B7AC270D8C3ED94FE601350CEBD00F4
:101CB00025EC60097520007521FF0200008100A855
:101CC00027A9280809D804D90281D3B17FEA89AAB3
:101CD000F281C50D81A0C3ED94035049EDA2E092BD
:101CE000007AC5C3E5829400E583941C50902000DF
:101CF00010438F02438F0175B7A575B7F1F030001F
:101D00001FA827A9280809438F01538FFDD804D99C
:101D100002A12089AAE275B7A575B7F1F0A3A10DBC
:101D2000538FFC817C7AC1BD030CE493A3FAB140CC
:101D3000DCF8B138817C817EAA22AB23B15CEBFA5E
:101D4000EA6222752608C3E52313F523E52213F57D
:101D50002250066323A0632201D526EAB1C9B1C986
:101D600075260AEAF4200102D287300102C287B147
:101D7000C9C3134002C201D526EB22B17FEAFB2082
:101D80008702A17F308702A184752608AE24AF2583
:101D9000C3EF13FFEE13FEB1CDB1C9C3EA13308711
:101DA000024480FA30E703632201C3E52313F523DD
:101DB000E52213F52250066323A0632201D526D91C
:101DC000E52265236523F52222AE24AF250E0FDE22
:101DD000FEDFFCD20122424C48656C693437316326
:041DE000F3300601D5
:00000001FF
